:100000000EC026C025C024C02AC022C021C020C0E6
:100010001FC01EC01DC01CC01BC01AC019C01124A7
:100020001FBECFEDCDBF10E0A0E6B0E0E8E5F1E007
:1000300002C005900D92A036B107D9F710E0A0E6F6
:10004000B0E001C01D92A936B107E1F704D082C02B
:10005000D7CF0895089557D0FCDFFCDFFECF1F9265
:100060000F920FB60F9211242F933F934F935F93EC
:100070006F937F938F939F93AF93BF93209164006F
:100080003091650040916600509167007091680062
:10009000DA01C9010296A11DB11D672F6A5F6D3794
:1000A00030F06D57DA01C9010396A11DB11D6093AF
:1000B00068008093640090936500A0936600B093FD
:1000C00067008091600090916100A0916200B09102
:1000D00063000196A11DB11D8093600090936100A3
:1000E000A0936200B0936300BF91AF919F918F91F5
:1000F0007F916F915F914F913F912F910F900FBE24
:100100000F901F901895789480B7806880BF80B753
:10011000806480BF8CB580648CBD8FEF8DBD80B74F
:10012000807F846080BF89B7846089BF83B7887F00
:1001300083BF8AB58C7F81608ABD83B7877F83BF89
:1001400083B7887F826083BF86B1887F836086B9EA
:08015000379A0895F894FFCFDF
:00000001FF
